:100000003FC10000F3C70000C6C7000099C7000049
:100010006CC700003FC7000012C7000062C10000AB
:1000200060C100005EC100005CC100005AC1000058
:1000300058C1000056C1000054C1000052C1000068
:1000400050C100004EC100004CC100004AC1000078
:1000500048C1000046C1000044C10000A6C600001F
:1000600040C100006CC6000041C600003AC100005B
:1000700038C1000036C1000034C1000032C10000A8
:1000800030C100002EC100002CC100002AC10000B8
:1000900028C1000026C1000024C1000022C10000C8
:1000A00020C100001EC100001CC100001AC10000D8
:1000B00018C1000016C1000014C1000012C10000E8
:1000C00010C100000EC100000CC100000AC10000F8
:1000D00008C1000006C1000004C1000002C1000008
:1000E00000C100002F0A002300230023005C23230B
:1000F00023235265616C53696D476561722300006B
:10010000002100240027002A002D003000330001C8
:10011000010000040107010A010000220025002857
:10012000002B002E00310034000201000005010800
:10013000010B01000020002300260029002C002FC5
:100140000032000001000003010601090105050558
:1001500005070508080808020202020A0A0808043E
:10016000040404010101010101010103030303036C
:10017000030303040707070C0C0C0C0C0C0C0C02FB
:1001800002020206060606060606060B0B0B0B0B02
:100190000B0B0B01021020200808102040102040FB
:1001A000800201020108040201010204081020403B
:1001B0008080402010080402018004020180402059
:1001C0001008040201080402010102040810204082
:1001D00080010204081020408000000A0B02090C74
:1001E0000D0E0807030401000000000000000000DD
:1001F00000000000000000000000000000000000FF
:1002000000000000001211100000000000000000BB
:100210000000000000000000000000000000002FAF
:100220000A002300230023005C232323235265615B
:100230006C53696D4765617223003D300A003D31A2
:100240000A000A003D300A003D310A003D300A0034
:100250003D310A003D300A003D310A000A000A0023
:100260002F0A002300230023005C2323232352654D
:10027000616C53696D47656172230000BD08F20E21
:1002800011241FBECFEFD1E2DEBFCDBF00E00CBF17
:100290002BE0AAE5B7E001C01D92AA38B207E1F74A
:1002A00017E0A0E0B2E0E6E2F3E200E00BBF02C03C
:1002B00007900D92AA35B107D9F711E0CFE3D1E04D
:1002C00000E006C021970109802FFE010E945D0F0A
:1002D000CE33D10780E00807A9F70E94350A0C94B5
:1002E00082118ECEAF92BF92CF92DF92EF92FF92A9
:1002F0000F931F93CF93DF936C017B018B01040F4E
:10030000151FEB015E01AE18BF08C017D10759F0E9
:100310006991D601ED91FC910190F081E02DC6012B
:100320001995892B79F7C501DF91CF911F910F9115
:10033000FF90EF90DF90CF90BF90AF900895E6EDE3
:10034000F8E0448155816081718180E398E0CACFF3
:10035000FC01538D448D252F30E0842F90E0821BCB
:10036000930B541710F0CF96089501970895FC0150
:10037000918D828D981761F0A28DAE0FBF2FB11DA8
:100380005D968C91928D9F5F9F73928F90E0089500
:100390008FEF9FEF0895FC01918D828D981731F0BA
:1003A000828DE80FF11D858D90E008958FEF9FEF0E
:1003B0000895FC01918D228D892F90E0805C9F4FE4
:1003C000821B91098F739927089580E398E0F1DFEC
:1003D00021E0892B09F420E0822F0895FC01A48DEF
:1003E000A80FB92FB11DA35ABF4F2C91848D90E057
:1003F00001968F739927848FA689B7892C93A0893A
:10040000B1898C91837080648C93938D848D9813C3
:1004100006C00288F389E02D80818F7D8083089556
:10042000EF92FF920F931F93CF93DF93EC0181E044
:10043000888F9B8D8C8D98131AC0E889F9898081EB
:1004400085FF15C09FB7F894EE89FF896083E8891E
:10045000F98980818370806480839FBF81E090E010
:10046000DF91CF911F910F91FF90EF900895F62E9D
:100470000B8D10E00F5F1F4F0F731127E02E8C8D37
:100480008E110BC00FB607FCFACFE889F98980817D
:1004900085FFF5CFCE01A2DFF2CFEB8DEC0FFD2F64
:1004A000F11DE35AFF4FF0829FB7F8940B8FEA8952
:1004B000FB8980818062D0CF0F931F93CF93DF930E
:1004C0008C01D0E0C0E0F801EC0FFD1F64916623C1
:1004D00039F080E398E0A4DF892B11F02196F3CF67
:1004E000CE01DF91CF911F910F910895CF93DF93AC
:1004F000EC01888D8823B1F0AA89BB89E889F98944
:100500008C9185FD03C0808186FD0CC00FB607FC71
:10051000F7CF8C9185FFF2CF808185FFEDCFCE01A3
:100520005DDFEACFDF91CF9108958150823108F0ED
:100530005AC0E82FF0E08827EF55FD4F8F4F0C94FD
:100540005D0FC102C502B302B902BD02F302C802C7
:10055000CE02D202D802DC02E002E602EA02F30294
:10056000EE02F402F802809180008F778093800081
:100570000895809180008F7DF9CF80918000877FE2
:10058000F5CF84B58F7784BD089584B58F7DFBCF7B
:100590008091B0008F778093B00008958091B00073
:1005A0008F7DF9CF809190008F7780939000089590
:1005B000809190008F7DF9CF80919000877FF5CF5B
:1005C0008091A0008F778093A00008958091A00073
:1005D0008F7DF9CF8091A000877FF5CF809120019A
:1005E0008F77809320010895809120018F7DF9CF2E
:1005F00080912001877FF5CFCF93DF93282F30E0C4
:10060000F901E752FE4F8491F901ED56FE4FD49166
:10061000F901E35BFE4FC491CC2399F0811185DF92
:10062000EC2FF0E0EE0FFF1FED5CFE4FA591B491B3
:10063000EC91ED2381E090E009F480E0DF91CF912F
:10064000089580E090E0FACF1F93CF93DF93282F97
:1006500030E0F901E752FE4F8491F901ED56FE4F6B
:10066000D491F901E35BFE4FC491CC23A1F0162F86
:1006700081115BDFEC2FF0E0EE0FFF1FE75EFE4F16
:10068000A591B4918FB7F894EC91111108C0D09551
:10069000DE23DC938FBFDF91CF911F910895DE2B76
:1006A000F8CFCF93DF9390E0FC01ED56FE4F2491FD
:1006B000835B9E4FFC0184918823C9F090E0880FF2
:1006C000991FFC01E150FF4FA591B491FC01E75E39
:1006D000FE4FC591D49161110DC09FB7F8948C91D4
:1006E000209582238C938881282328839FBFDF91C4
:1006F000CF910895623051F49FB7F8943C91822FC6
:10070000809583238C93E8812E2BEFCF8FB7F894BD
:10071000EC912E2B2C938FBFEACF3FB7F8948091AA
:10072000D1079091D207A091D307B091D40726B5F5
:10073000A89B05C02F3F19F00196A11DB11D3FBF19
:10074000BA2FA92F982F8827BC01CD01620F711DE8
:10075000811D911D42E0660F771F881F991F4A95E2
:10076000D1F708958F929F92AF92BF92CF92DF926E
:10077000EF92FF924B015C01D0DF6B017C01CDDF7A
:100780006C197D098E099F09683E734081059105AA
:10079000B0F321E0821A9108A108B10888EEC80ED2
:1007A00083E0D81EE11CF11C81149104A104B10462
:1007B00031F7FF90EF90DF90CF90BF90AF909F9078
:1007C0008F9008952FB7F8946091CD077091CE0760
:1007D0008091CF079091D0072FBF0895FC018481AD
:1007E00087FD04C091E0692763832EDF80E00895D0
:1007F000EF92FF921F93CF93DF93EC01E62E062E2C
:10080000000CFF088A81082E000C990BE816F906E7
:10081000A1F06A8310E08985181778F4B701012EDA
:1008200002C0759567950A94E2F76170FE01E10FC9
:10083000F11D858109DF1F5FEECF8C85882329F0AC
:10084000813049F18FEF9FEF20C08B85863308F010
:10085000865320917B00982F9870277F922B90933E
:100860007B008770806480937C0080917A00806434
:1008700080937A0080917A0086FDFCCF9091780079
:1008800080917900892798278927DF91CF911F913F
:10089000FF90EF9008958B85DF91CF911F91FF908E
:1008A000EF90AACEFC01808580FD04C082FB8827E2
:1008B00080F9089580E00895FC019085957081E0AD
:1008C000953009F080E00895862F642FEACEFC0170
:1008D000818592DE21E0892B09F420E0822F0895A2
:1008E000DC01ED91FD918081ED91FD919081ED9183
:1008F000FD916C9163708E2309F064609F2309F071
:100900006860EDE8F4E0E60FF11D659565956D937F
:100910006D917D918D919D91099423C01AC012C053
:1009200016C010C01EC009C014C013C006C019C034
:1009300009C00DC007C00DC014C062507040804097
:1009400090400BC0615070408040904006C06E5F88
:1009500001C06F5F7F4F8F4F9F4F9E938E937E930B
:100960006E930895CF93DF93EC018B85823058F41A
:10097000F894CE01B5DF6F81788589859A85789462
:10098000DF91CF910895F894F6CF8F929F92AF9216
:10099000BF920F931F93CF93DF93CDB7DEB7A1978D
:1009A0000FB6F894DEBF0FBECDBF19A2423008F4D7
:1009B0004AE08E010F5D1F4F842E912CB12CA12C8B
:1009C000A50194010E941F0FE62FB901CA01EA3068
:1009D0003CF5E05DD801EE938D01232B242B252BD4
:1009E00079F790E080E0109761F0FD010190002020
:1009F000E9F73197AF014A1B5B0BBD0180E398E03B
:100A000071DCA1960FB6F894DEBF0FBECDBFDF91AB
:100A1000CF911F910F91BF90AF909F908F900895AD
:100A2000E95CD8CF4AE061E070E080E090E0ADCFD3
:100A3000009761F0FC0101900020E9F73197AF01C8
:100A4000481B590BBC0180E398E04CCC90E080E05F
:100A500008950F931F93CF93DF9380E398E0A9DC71
:100A6000892B09F44EC080E398E081DC8C37C1F417
:100A70008DEE90E021DD82E393E0DADF8BEE90E013
:100A80001BDDD0DF89EE90E017DD8EE092E0D0DF55
:100A900087EE90E011DD53DC84EE90E00DDDDDCFDC
:100AA0008C3329F41092CB071092CA07D6CF8A3024
:100AB000B1F4CEE1D2E006E617E089919991009772
:100AC00039F0F801208161E0213309F060E0BCDDFC
:100AD0000F5F1F4FF2E0C033DF0779F7E3CF2091BC
:100AE000CA073091CB0724363105E4F6F901EA59FB
:100AF000F84F80832F5F3F4F3093CB072093CA0777
:100B0000ACCFDF91CF911F910F9108955EDC8111E1
:100B1000A0DF80E090E0892B49F080E090E0892B15
:100B200029F00E94000081110E94000080E090E006
:100B3000892B49F080E090E0892B29F00E94000089
:100B400081110E94000080E090E0892B49F080E054
:100B500090E0892B29F00E94000081110C94000084
:100B60000895CF92DF92EF92FF920F931F93CF934E
:100B7000DF93EC01E62E84E090E00E94650FFC011B
:100B800082E0808383E0818394E0928385E08383A5
:100B900020E133E0398328838FEF8A838B838C8332
:100BA0008A878B878C8799878F016E0185E0C80EB5
:100BB000D11CF12CF80181918F0187FD32C0F60123
:100BC00081936F0161E06DDDF394F4E0FF12F2CFE9
:100BD0008FEF8C8386E193E0998388838B8587FDF3
:100BE0000FC0282F082E000C330BE216130641F01D
:100BF0009A85913011F460E027DD60E08B8551DD4E
:100C000082E08A87EB8662E08E2D4BDD81E08C8767
:100C1000DF91CF911F910F91FF90EF90DF90CF90D8
:100C20000895F986D5CFCF93DF93EC018881998120
:100C3000009711F00E940110198218821D821C82F7
:100C40001B821A82DF91CF910895FC0180819181EE
:100C5000009711F00C94011008950E9466110F93F3
:100C60001F93CF93DF93EC0188819981009759F00E
:100C70002A813B812617370730F081E0DF91CF9141
:100C80001F910F9108958B016F5F7F4F0E948A1013
:100C9000009759F0998388831B830A832C813D81B7
:100CA000232B59F7FC011082E8CF80E0E7CFEF92C9
:100CB000FF920F931F93CF93DF93EC017B018A0187
:100CC000BA01CDDF81110AC0CE01ADDFCE01DF91C7
:100CD000CF911F910F91FF90EF9008951D830C838A
:100CE000B701888199810E947B11F0CF1F920F92EA
:100CF0000FB60F9211240BB60F922F933F934F9381
:100D00005F936F937F938F939F93AF93BF93EF9373
:100D1000FF9380E398E062DBFF91EF91BF91AF9189
:100D20009F918F917F916F915F914F913F912F9103
:100D30000F900BBE0F900FBE0F901F9018951F9233
:100D40000F920FB60F9211240BB60F922F938F9321
:100D50009F93EF93FF93E0914008F09141088081C9
:100D6000E0914608F091470882FD1DC09081809176
:100D700049088F5F8F7320914A08821741F0E091F4
:100D80004908F0E0E05DF74F958F80934908FF91A7
:100D9000EF919F918F912F910F900BBE0F900FBEEF
:100DA0000F901F9018958081F2CF1F920F920FB66F
:100DB0000F9211242F933F938F939F93AF93BF93E1
:100DC0008091CD079091CE07A091CF07B091D00729
:100DD0003091CC0723E0230F2D3758F50196A11D44
:100DE000B11D2093CC078093CD079093CE07A0939D
:100DF000CF07B093D0078091D1079091D207A091EF
:100E0000D307B091D4070196A11DB11D8093D107DE
:100E10009093D207A093D307B093D407BF91AF911B
:100E20009F918F913F912F910F900FBE0F901F9028
:100E3000189526E8230F0296A11DB11DD2CF1F924F
:100E40000F920FB60F9211240BB60F922F933F9370
:100E50004F935F936F937F938F939F93AF93BF93C2
:100E6000EF93FF9380915C0790915D0739DDFF91CF
:100E7000EF91BF91AF919F918F917F916F915F9112
:100E80004F913F912F910F900BBE0F900FBE0F907F
:100E90001F9018951F920F920FB60F9211240BB648
:100EA0000F922F933F934F935F936F937F938F9303
:100EB0009F93AF93BF93EF93FF9380915A079091C5
:100EC0005B070EDDFF91EF91BF91AF919F918F91E5
:100ED0007F916F915F914F913F912F910F900BBE3A
:100EE0000F900FBE0F901F9018951F920F920FB684
:100EF0000F9211240BB60F922F933F934F935F9352
:100F00006F937F938F939F93AF93BF93EF93FF93D1
:100F10008091640790916507E3DCFF91EF91BF91A9
:100F2000AF919F918F917F916F915F914F913F9181
:100F30002F910F900BBE0F900FBE0F901F90189522
:100F40001F920F920FB60F9211240BB60F922F9390
:100F50003F934F935F936F937F938F939F93AF9341
:100F6000BF93EF93FF938091620790916307B8DC82
:100F7000FF91EF91BF91AF919F918F917F916F9171
:100F80005F914F913F912F910F900BBE0F900FBE2D
:100F90000F901F9018951F920F920FB60F92112469
:100FA0000BB60F922F933F934F935F936F937F9363
:100FB0008F939F93AF93BF93EF93FF9380916007BD
:100FC000909161078DDCFF91EF91BF91AF919F915F
:100FD0008F917F916F915F914F913F912F910F90E2
:100FE0000BBE0F900FBE0F901F9018951F920F927F
:100FF0000FB60F9211240BB60F922F933F934F937E
:101000005F936F937F938F939F93AF93BF93EF9370
:10101000FF9380915E0790915F0762DCFF91EF91F3
:10102000BF91AF919F918F917F916F915F914F9100
:101030003F912F910F900BBE0F900FBE0F901F90FE
:10104000189590E0823090F404968330910569F110
:101050007CF481309105C9F00297F9F08091690024
:101060008C7F816080936900E89A08950297EDCFA4
:101070008430910511F1059789F780916A00837F8B
:10108000846080936A00ED9A089580916900837F5F
:10109000846080936900E99A0895809169008F7C4B
:1010A000806180936900EA9A0895809169008F7346
:1010B000806480936900EB9A089580916A008C7F28
:1010C000816080936A00EC9A089580E008950F9300
:1010D0001F93CF93DF93EC01062F142F62E0802F34
:1010E000E0DA62E0812FDDDA802F90E0FC01E35B43
:1010F000FE4FE491F0E0EE0FFF1FED5CFE4FA59177
:10110000B491B983A883FC01ED56FE4F24912C8342
:10111000812F90E0FC01E35BFE4FE491F0E0EE0FE5
:10112000FF1FED5CFE4F459154915B834A83FC01A8
:10113000ED56FE4FE491ED831F82188619861A86BC
:101140008BE39FE10197F1F78C91282391E009F45B
:1011500090E0DA018C91E82309F092609E83BE0151
:10116000802FB3DF082FBE01812FAFDF800F8B8769
:10117000DF91CF911F910F91089510923308109233
:10118000320888EE93E0A0E0B0E0809334089093BA
:101190003508A0933608B09337088CE193E090931C
:1011A00031088093300885EC90E090933D0880935F
:1011B0003C0884EC90E090933F0880933E0880ECDC
:1011C00090E0909341088093400881EC90E09093E8
:1011D00043088093420882EC90E090934508809306
:1011E000440886EC90E0909347088093460810925C
:1011F000490810924A0810924B0810924C08ADEC26
:10120000B8E090E080E041E2FC013E9621E030E071
:101210008630910510F430E020E0E20FF31F409398
:101220005700E491ED9301968930910569F766E0E6
:1012300089E79BE096DC67E08CE69BE092DC4DE280
:101240006CE28CE89AE043DF87E493E09093990A9C
:101250008093980A88E593E090939B0A80939A0A7A
:101260004EE26FE28CE99AE032DF89E693E09093F8
:10127000A90A8093A80A8AE793E09093AB0A809327
:10128000AA0A4AE26BE28CEA9AE021DF8BE893E05B
:101290009093B90A8093B80A8CE993E09093BB0AC3
:1012A0008093BA0A49E268E28CEB9AE010DF8DEA9B
:1012B00093E09093C90A8093C80A8EEB93E09093D1
:1012C000CB0A8093CA0A40E361E38CEC9AE0FFDE2C
:1012D0008FEC93E09093D90A8093D80A8AED93E03B
:1012E0009093DB0A8093DA0A4FE16EE18CED9AE08D
:1012F000EEDE85EE93E09093E90A8093E80A82EFB0
:1013000093E09093EB0A8093EA0A45E264E28CEE64
:101310009AE0DDDE8FEF93E09093F90A8093F80A6C
:1013200080E194E09093FB0A8093FA0A46E267E238
:101330008CEF9AE0CCDE81E294E09093090B8093ED
:10134000080B82E394E090930B0B80930A0B43E22B
:1013500062E28CE09BE0BBDE83E494E09093190BA7
:101360008093180B8EE494E090931B0B80931A0BE0
:1013700041E260E28CE19BE0AADE89E594E0909393
:10138000290B8093280B85E694E090932B0B809398
:101390002A0B48E169E18CE29BE099DE81E794E069
:1013A0009093390B8093380B82E894E090933B0B39
:1013B00080933A0B47E166E18CE39BE088DE83E9AA
:1013C00094E09093490B8093480B84EA94E09093C7
:1013D0004B0B80934A0B43E362E38CE49BE077DEA4
:1013E00085EB94E09093590B8093580B84EC94E038
:1013F00090935B0B80935A0B45E364E38CE59BE091
:1014000066DE83ED94E09093690B8093680B82EE27
:1014100094E090936B0B80936A0BECEDF8E02EE276
:1014200033E08AE090E031832083128213821482B9
:101430001582978386831086118672964AE0EC386F
:10144000F40789F71092D7081092D6081092D9089D
:101450001092D8081092DB081092DA0850E040E0B1
:1014600063E075E086ED98E022CCCF93DF93CDB7B3
:10147000DEB760970FB6F894DEBF0FBECDBF78948D
:1014800084B5826084BD84B5816084BD85B5826089
:1014900085BD85B5816085BD80916E00816080933A
:1014A0006E001092810080918100826080938100A3
:1014B00080918100816080938100809180008160B3
:1014C000809380008091B10084608093B10080910E
:1014D000B00081608093B000809191008260809321
:1014E00091008091910081608093910080919000A3
:1014F0008160809390008091A10082608093A10020
:101500008091A10081608093A1008091A000816002
:101510008093A000809121018260809321018091BD
:10152000210181608093210180912001816080935D
:10153000200180917A00846080937A0080917A0003
:10154000826080937A0080917A00816080937A0033
:1015500080917A00806880937A001092C100E091B7
:101560004008F091410882E08083E0913C08F091CE
:101570003D081082E0913E08F0913F0880E18083B1
:1015800010924808E0914408F091450886E0808375
:10159000E0914208F0914308808180618083E0916E
:1015A0004208F0914308808188608083E09142087E
:1015B000F0914308808180688083E0914208F09137
:1015C000430880818F7D808382E390E0A0E0B0E0DB
:1015D0008093340890933508A0933608B093370869
:1015E00068EE73E080E090E0BDD80EECC02E08E01D
:1015F000D02E8E010F5F1F4FD6018D916D011B867E
:101600001A861D861C861F861E8640E1B80190E062
:10161000EDD3F80101900020E9F73197AF01401BAD
:10162000510BB801CE010A9642DB1A8219821C8244
:101630001B821E821D826091D6087091D7086115A9
:10164000710531F04091DA085091DB08C8012FDBB9
:101650008E859F85AA84BB84ED80FE80E80EF91EEE
:10166000A114B10409F439C0892B79F0B701C8017C
:10167000F6DA882391F129813A818D819E81B50125
:10168000820F931F38D6FE82ED8269817A816115BF
:10169000710531F14D815E8186ED98E008DBC8016E
:1016A000D4DACE010A96D1DAB6EDCB16B8E0DB0675
:1016B00009F0A2CF0091D6081091D70801151105A5
:1016C00099F0F8018081882379F0082E000C990B9D
:1016D00001D6D8018D938D01F4CFC801A4DAD5CFFE
:1016E00086ED98E0A0DADBCF88E292E00E945C020F
:1016F00082E393E09DD986E292E00E945C0292D957
:1017000084E292E00E945C028EE092E091D982E253
:1017100092E00E945C020E949F018FE192E00E9491
:101720005C0215EEE12E17E0F12E10E0612F89E743
:101730009BE05ED8F70181937F011F5F1F30B1F7F7
:10174000B5EDEB2EB7E0FB2E10E0612F8CE69BE0B1
:101750004FD8D7018D937D011F5F1031B1F70CED8C
:1017600018E0FCEAEF2EF2E0FF2EAAE0AA2EB12C40
:10177000F701D0807181D801ED91FC910280F38155
:10178000E02D42E050E06D2DC8011995F801D18699
:1017900010860190F081E02D0190F081E02DC801CC
:1017A0001995882339F0D80118968C911897836081
:1017B00018968C9307D8F80162837383848395838A
:1017C000B782A682F4E0EF0EF11C0E5E1F4F4AE0D6
:1017D0000C38140769F608EF17E0ECE8EE2EEAE0A3
:1017E000FE2EC701BFD8D8016D937D938D939D9335
:1017F0008D01B0E1EB0EF11CE8E000331E0789F724
:101800000EE112E07801D701CD90DD907D01C11489
:10181000D10441F061E08C2D0E94510361E08C2DD8
:101820000E942403B0E3EB16B2E0FB0661F768EB1D
:101830007BE080E090E00E94B203F80181919191F9
:101840008F01009719F060E00E942403F2E000335A
:101850001F0799F772E3272E73E0372E0E94E203E9
:101860004B015C018091140290911502A091160227
:10187000B0911702AC01BD014854544F6F4F7F4FD8
:1018800084169506A606B70628F488169906AA06B1
:10189000BB0668F589E692E00E945C0282E393E071
:1018A000C7D887E692E00E945C02BCD885E692E049
:1018B0000E945C028EE092E0BBD883E692E00E9438
:1018C0005C020E949F0180E692E00E945C0280928E
:1018D000140290921502A0921602B0921702809202
:1018E0000A0290920B02A0920C02B0920D0268EFD5
:1018F000E62E67E0F62E0CE81AE091E041EF2416A0
:1019000044E0340609F090E0D8011C962D913C91FA
:10191000B3E02F3C3B0709F4B5C12450354009F42E
:10192000B1C1D8011E962D913C9181E0B3E02A3DD2
:101930003B0721F02F50354009F080E0992309F44E
:10194000A3C1882309F4A0C1C8010CD824E030E069
:1019500040E050E096D229013A01F701808191815F
:10196000A281B38184159505A605B7050CF094C135
:10197000D8011E968D919C915BD88EE592E00E94D5
:101980005C0280920A0290920B02A0920C02B0922A
:101990000D02D7014D925D926D927D927D01005FA7
:1019A0001F4FECE6FBE0E017F10709F0A6CF5CEA79
:1019B000C52E52E0D52E0CED18E0F12CE12CD8010B
:1019C00018968C9118978B7F18968C931897ED9199
:1019D000FC910190F081E02DC8011995888BF801E8
:1019E0008085869581704888481609F463C10E94F5
:1019F000E203D80112966D937D938D939C93159776
:101A000018968C91B2E08B27F8018087C8010E945C
:101A10005204811106C0C8010E945C04882309F4A5
:101A2000C2C131E0BAE12B16B5E03B0609F030E067
:101A3000F60180819181AC014B7F21E04332510559
:101A400039F08B32910521F08D32910509F020E0BB
:101A5000332311F021117EC1AC01435151094330B0
:101A6000510508F477C18C31910509F473C18532B1
:101A7000910509F0A6C1332309F4A3C180910602A0
:101A800090910702A0910802B091090283589F4FDC
:101A9000AF4FBF4F88169906AA06BB0630F181E00A
:101AA00090E09093F7078093F607F092F507E092A5
:101AB000F4078092020290920302A0920402B09274
:101AC0000502C8010E945204882321F010920102ED
:101AD00010920002C8010E945C04882331F081E06A
:101AE00090E0909301028093000261E070E080E05A
:101AF00090E00E94B20300E712E045EEE42E47E0DA
:101B0000F42ED12C6D2D89E79BE00E94F803C82E9E
:101B1000D7018D917D01C81699F0FD013197C082E2
:101B2000F801828193810E94180580E592E0CC2023
:101B300029F0F1E0CF1204C08CE492E00E945C0234
:101B4000D3940C5F1F4F3FE0432ED410DBCF00E354
:101B500012E025EDE22E27E0F22ED12C6D2D8CE641
:101B60009BE00E94F803C82ED7018D917D01C81615
:101B700099F0FD013197C082F801828193810E9422
:101B8000180588E492E0CC2029F0F1E0CF1204C0DF
:101B900084E492E00E945C02D3940C5F1F4F90E1BA
:101BA000492ED410DBCF80910A0290910B02A091B4
:101BB0000C02B0910D02AC01BD014C595F4F6F4F4B
:101BC0007F4F84169506A606B70628F48816990650
:101BD000AA06BB0660F482E492E00E945C02809256
:101BE0000A0290920B02A0920C02B0920D02809118
:101BF000020290910302A0910402B0910502835861
:101C00009F4FAF4FBF4F88159905AA05BB05B8F583
:101C10008091F6079091F707019789F5E091F40715
:101C2000F091F507EE0FFF1FEE0FFF1FE455FD4F7C
:101C3000828193810E941805809100029091010297
:101C4000009709F0C9C08EE392E00E945C0264E64E
:101C500070E080E090E00E94B20380920A029092CD
:101C60000B02A0920C02B0920D021092F707109294
:101C7000F60789E090E090930102809300020E94B1
:101C80008605ECCD81E05ACEC8010E94B20422E064
:101C900030E040E050E05ECE481659066A067B060A
:101CA0000CF077CEF801848595850E9418058CE5A7
:101CB00092E065CE0E94E203D80112962D913D91EB
:101CC0004D915C9115972B013C01421A530A640A0D
:101CD000750AB301A20116968D919C91B0E0A0E027
:101CE000481759076A077B0708F490CED801189661
:101CF0008C9181704888481609F488CE0E94E203CE
:101D0000D80112966D937D938D939C931597189699
:101D10008C91B1E08B278460F80180870E94E203F8
:101D2000D8011A964D905D906D907C901D97641926
:101D3000750986099709F80166877787808B918BEB
:101D40000E94E203D8011A966D937D938D939C9324
:101D50001D975CCE8092060290920702A092080224
:101D6000B09209021092F7071092F607D601129668
:101D70008D919C910E941805C8010E9452048823ED
:101D800019F188E592E00E945C0264E670E080E070
:101D900090E00E94B20380920A0290920B02A092FD
:101DA0000C02B0920D02BFEFEB1AFB0A0E5E1F4F42
:101DB000E4E0CE0ED11CF8E1EF16F10409F0FFCDFE
:101DC00094CE4A9799F65ACEC8010E945C048823A3
:101DD000E1F284E592E0D7CF019709F038CF8AE3AA
:101DE00092E033CF86ED98E00C942506BB27FB01EB
:101DF0005527AA27880F991FAA1FA41710F0A41B04
:101E000083955051B9F7A05DAA3308F0A95DA1935D
:101E1000009779F7B111B1931192CB0100C0DC01A9
:101E2000FC01672F71917723E1F7329704C07C9111
:101E30006D9370836291AE17BF07C8F30895A1E256
:101E40001A2EAA1BBB1BFD010DC0AA1FBB1FEE1F34
:101E5000FF1FA217B307E407F50720F0A21BB30B7F
:101E6000E40BF50B661F771F881F991F1A9469F7FB
:101E700060957095809590959B01AC01BD01CF0157
:101E80000895052E97FB16F400940FD057FD05D04A
:101E9000D6DF07FC02D046F408C050954095309537
:101EA00021953F4F4F4F5F4F0895909580957095C6
:101EB00061957F4F8F4F9F4F0895EE0FFF1F881F33
:101EC0008BBF0790F691E02D19940F931F93CF933A
:101ED000DF938230910510F482E090E0E091880B6E
:101EE000F091890B30E020E0B0E0A0E0309799F469
:101EF0002115310509F44AC0281B390B243031055E
:101F0000D8F58A819B816115710589F1FB01938365
:101F10008283FE0111C040815181028113814817E3
:101F20005907E0F04817590799F4109761F0129695
:101F30000C93129713961C933296CF01DF91CF9199
:101F40001F910F9108950093880B1093890BF4CF84
:101F50002115310551F04217530738F0A901DB0173
:101F60009A01BD01DF01F801C1CFEF01F9CF9093D4
:101F7000890B8093880BCDCFFE01E20FF31F819375
:101F800091932250310939832883D7CF2091860B32
:101F90003091870B232B41F420911A0230911B02C0
:101FA0003093870B2093860B2091180230911902F1
:101FB0002115310541F42DB73EB740911C025091D7
:101FC0001D02241B350BE091860BF091870BE21765
:101FD000F307A0F42E1B3F0B2817390778F0AC014C
:101FE0004E5F5F4F2417350748F04E0F5F1F509329
:101FF000870B4093860B819391939FCFF0E0E0E0B5
:102000009CCFCF93DF930097E9F0FC0132971382C6
:102010001282A091880BB091890BED0130E020E095
:102020001097A1F420813181820F931F2091860B9C
:102030003091870B2817390709F061C0F093870B9F
:10204000E093860BDF91CF910895EA01CE17DF0769
:10205000E8F54A815B819E0141155105B1F7E9011F
:10206000FB83EA8349915991C40FD51FEC17FD07F3
:1020700061F4808191810296840F951FE901998313
:102080008883828193819B838A83F0E0E0E01296CB
:102090008D919C9113970097B9F52D913C911197D3
:1020A000CD010296820F931F2091860B3091870BF2
:1020B0002817390739F6309751F51092890B10928D
:1020C000880BB093870BA093860BBCCFD383C283BE
:1020D00040815181840F951FC817D90761F44E5F65
:1020E0005F4F88819981480F591F518340838A81AE
:1020F0009B81938382832115310509F0B0CFF09342
:10210000890BE093880B9ECFFD01DC01C0CF1382C9
:102110001282D7CF4F925F926F927F928F929F924F
:10212000AF92BF92CF92DF92EF92FF920F931F93E5
:10213000CF93DF938C01009791F4CB01DF91CF9186
:102140001F910F91FF90EF90DF90CF90BF90AF90D5
:102150009F908F907F906F905F904F90B6CEFC01D4
:10216000E60FF71F9C0122503109E217F30708F42C
:10217000AAC0D901CD91DC911197C617D70718F1E4
:10218000C530D10570F0CE0104978617970748F047
:10219000C61BD70B2297C193D1936D937C93CF012C
:1021A00030DFC801DF91CF911F910F91FF90EF9029
:1021B000DF90CF90BF90AF909F908F907F906F9067
:1021C0005F904F9008955B01AC1ABD0A4C018C0ED4
:1021D0009D1EA091880BB091890B512C412CF12CA4
:1021E000E12C109731F58091860B9091870B881523
:1021F000990509F05CC04616570608F058C0809152
:10220000180290911902009741F48DB79EB7409142
:102210001C0250911D02841B950BE817F90708F06A
:1022200052C0F093870BE093860BF90171836083B2
:10223000B8CF8D919C91119712966C90129713962E
:102240007C901397A815B90559F56C0142E0C40EAE
:10225000D11CCA14DB0420F1AC014A195B09DA0174
:102260001296159780F06282738251834083D90160
:102270006D937C93E114F10471F0D7011396FC93F4
:10228000EE9312978ECF22968C0F9D1FF9019183AA
:102290008083F301EFCFF093890BE093880B81CF1C
:1022A0004816590608F42C017D01D3019ACFCB01C1
:1022B0000CDE7C01009739F0AE01B80113D0C801E3
:1022C000A0DE87016ECF10E000E06BCF81E090E0F0
:1022D000F89418C09111089581568A5108F48052DB
:1022E00085580895FB01DC0102C001900D92415018
:1022F0005040D8F70895FB01DC0101900D920020B9
:10230000E1F7089511E0CFE3D1E000E005C0802FB0
:10231000FE01D3DD2196011DC034D10780E00807FE
:06232000B1F7F894FFCFB5
:102326000900FFFFFFFFFFFFFFFFFFFFFFFF332E49
:10233600312E3900FFFFFFFF00008A0B80000900E5
:102346000A000B00080010000F000C000D000E0024
:1023560000002A050100330502003B050300440581
:1023660004004C050500550506005E0507006605D8
:1023760008006F05090078050A0086050B008E0522
:102386000C0096050D00A1050E00A9050F00B2056B
:102396000000BB050100C7050200D2050300DD05EC
:1023A6000400EA050500F6050600020607000E060B
:1023B60008001906090024060A002F060B003A0633
:1023C6000C0045060D0051060E005D061500690657
:1023D6001C0074061300820614008D061A009A0665
:1023E6001100A7061B00B3061200BB063600C8067E
:1023F6003C00CF063700D6063D00DE063800E6066E
:102406003E00EE063900F7063F00FF063A000607D3
:1024160040000D073B0019074100210742002D0728
:10242600430038074400430745004E0700000000FC
:102436002D0600000000EE030000000010027201ED
:10244600A8017602D901B701CB010000000067049C
:1024560064045265616C53696D476561722D47313D
:1024660030303058464400454E435F414C545F4F30
:10247600555445525F555000454E435F414C545F9D
:102486004F555445525F444E00454E435F414C54B0
:102496005F494E4E45525F555000454E435F414C95
:1024A600545F494E4E45525F444E00454E435F4E83
:1024B60041565F494E4E45525F555000454E435F6B
:1024C6004E41565F494E4E45525F444E00454E437F
:1024D6005F4E41565F4F555445525F555000454E2D
:1024E600435F4E41565F4F555445525F444E00453B
:1024F6004E435F4844475F555000454E435F48444E
:10250600475F444E00454E435F52414E47455F4448
:102516004E00454E435F52414E47455F555000457C
:102526004E435F434F4D5F4F555445525F555000E4
:10253600454E435F434F4D5F4F555445525F444EA2
:1025460000454E435F434F4D5F494E4E45525F55E2
:102556005000454E435F434F4D5F494E4E45525FD7
:10256600444E00454E435F4352535F555000454E1F
:10257600435F4352535F444E00454E435F424152D0
:102586004F5F555000454E435F4241524F5F444EA8
:1025960000454E435F464D535F4F555445525F5578
:1025A6005000454E435F464D535F4F555445525F6D
:1025B600444E00454E435F464D535F494E4E45528D
:1025C6005F555000454E435F464D535F494E4E455D
:1025D600525F444E00454E435F4E41565F564F4C48
:1025E6005F444E00454E435F4E41565F564F4C5F2B
:1025F600555000454E435F434F4D5F564F4C5F4429
:102606004E00454E435F434F4D5F564F4C5F55500E
:10261600005265616C53696D476561722D4746438B
:1026260035303000454E435F414C545F55500045B0
:102636004E435F414C545F444E005265616C536992
:102646006D476561722D4743550042544E5F4D49B3
:1026560043320042544E5F444D450042544E5F4D56
:102666004943310042544E5F4144460042544E5F56
:102676004E4156310042544E5F4E4156320042544E
:102686004E5F4D4B520042544E5F434F4D31004218
:10269600544E5F434F4D320042544E5F52455645AD
:1026A6005253494F4E0042544E5F434C52004254DF
:1026B6004E5F46504C0042544E5F44495245435487
:1026C6000042544E5F454E540042544E5F50524FA6
:1026D600430042544E5F4D454E550042544E5F41B5
:1026E6004C545F53454C0042544E5F434F4D5F463A
:1026F600460042544E5F4E41565F46460042544E97
:102706005F4844475F53594E430042544E5F4E4123
:10271600565F564F4C0042544E5F434F4D5F564FE7
:102726004C0042544E5F534F46545F313000425482
:102736004E5F534F46545F390042544E5F534F46E7
:10274600545F380042544E5F534F46545F37004241
:10275600544E5F534F46545F360042544E5F534FBC
:1027660046545F350042544E5F534F46545F3131F5
:102776000042544E5F534F46545F31320042544E2E
:102786005F4E41565F544F470042544E5F50414E94
:102796005F444E0042544E5F50414E5F5249474897
:1027A600540042544E5F50414E5F55500042544EC5
:1027B6005F50414E5F4C4546540042544E5F504177
:1027C6004E5F53594E430042544E5F434F4D5F5444
:1027D6004F470042544E5F464D530042544E5F43AE
:1027E60052535F53594E430042544E5F415000428C
:1027F600544E5F46440042544E5F4844470042549C
:102806004E5F414C540042544E5F4E415600425476
:102816004E5F564E41560042544E5F415052004262
:10282600544E5F42430042544E5F56530042544E4C
:102836005F4E4F53455F55500042544E5F464C43E2
:102846000042544E5F4E4F53455F444E0042544E35
:102856005F534F46545F310042544E5F534F4654C8
:102866005F320042544E5F534F46545F330042542A
:0A2876004E5F534F46545F340000DC
:00000001FF
